:1000000012C0189518951895189518951895189563
:100010001895189518951895189518951895189578
:100020001895189518958FED8DBFC0ECE8EB4E2E06
:10003000DD275D2EEEE7F0E0A0E6B0E088278D93A7
:100040003197E9F7662480EF87BB8FE881BB80E0BA
:1000500088BB80E082BBC39AC29AC19AC09A969A22
:10006000959A949AC79AC69A0027A0E38C9186FB2A
:100070000EF401E040E0041709F003C0E1E0F0E015
:100080009ED00027A0E38C9186FB0EF401E041E0B6
:10009000041709F005C0EEE1F0E091D0C69801C068
:1000A000E3CF0027A0E38C9185FB0EF401E041E053
:1000B000041709F007C020D0A0E6EC91FF277FD0FD
:1000C000C7985AD00027A0E38C9184FB0EF401E07E
:1000D00041E0041709F002C0C7984ED00027A0E302
:1000E0008C9186FB0EF401E040E0041709F003C098
:1000F000C69AC79AB9CFD5CF80E080936000002719
:10010000A6E38C9183FB0EF401E040E0041709F0B4
:1001100004C0A0E68C918E5F8C930027A6E38C919F
:1001200082FB0EF401E040E0041709F004C0A0E6F1
:100130008C918C5F8C930027A6E38C9181FB0EF44D
:1001400001E040E0041709F004C0A0E68C918A5F4A
:100150008C930027A6E38C9180FB0EF401E040E035
:10016000041709F004C0A0E68C91885F8C93A0E688
:100170008C918F5F8C930895C59A80E08093610085
:1001800000916100073710F009F017C00027A0E3C5
:100190008C9186FB0EF401E040E0041709F004C0E6
:1001A000C69AC79AC59860CFE1E0F0E008D0A1E612
:1001B0008C918F5F8C9308F4E3CFC598089588EEF7
:1001C00093E00CD03197D9F708953197F1F708955E
:1001D000689462F80895E89462F80895EF93FF93A5
:1001E000EE27E82BE92B31F0EAEFF0E03197F1F759
:0A01F0000197D1F7FF91EF910895F8
:00000001FF
